:100000000C94B7060C94D4060C94D4060C94D40625
:100010000C94D4060C94D4060C94D4060C94D406F8
:100020000C94D4060C94D4060C94262C0C94F82C26
:100030000C9439260C94D4060C94D4060C94D40653
:100040000C94D4060C94D4060C94D4060C94D406C8
:100050000C94D4060C94C1260C94D4060C94D406AB
:100060000C94D4060C94D4060C94D4060C94D406A8
:100070000C94D4060C94D4060C94D4060C94D40698
:100080000C94D4060C94D4060C94D4060C94D40688
:100090000C94D4060C94D4060C94D4060C94D40678
:1000A0000C94D4060C94D4060C94D4068D087E08C7
:1000B0008A0882088A088A088A0886088A088A08BC
:1000C0008A088A088A088A088A088A087C088008B8
:1000D0008A0884088A088A088A088808B60DB60D36
:1000E000E20DE20D4A0E680E800F800F730E0C0FAA
:1000F0001D0F1D0F662254226D22DF211A231A23A1
:1001000051221A231A239A221A23AE22FA221A23E0
:100110001A231A231A23CE221A231A23CB221A2394
:1001200086221A231A23142314231423142314239A
:10013000142314231423142316231A23662249227A
:100140001A231A231A231A231A231A231A231A23C7
:100150001A231A2316231A231A2351221A2312238D
:1001600012231223122312231223122312231223E7
:100170001623652D8C2D842E8C2D842ED82DFB2DB1
:10018000842E522E612E25733A2025642070656ED0
:1001900064696E67206B6579732061726520616D9B
:1001A000626967756F75730A0025733A206C6F6F0B
:1001B00070696E67207468726F75676820256420A7
:1001C0006B6579732E2E2E0A0025733A20676F74A3
:1001D000206475616C2D726F6C65206B65790A0007
:1001E00025733A2068616E646C65642062792071C1
:1001F0006D6B0A002025733A2063616E27742064BA
:100200006973616D626967756174652028796574C9
:10021000290A002025733A20666F756E6420737575
:100220006273657175656E7420646F776E7570208A
:10023000706169722C20696E746572707265746980
:100240006E672068656164206173206D6F640A00C9
:100250002025733A20666F756E6420646F776E2D6B
:10026000757020706169722C20696E74657270728D
:100270006574696E67206173206E6F726D616C20AA
:100280006B65790A002025733A20696E7465727077
:10029000726574696E67206B657975702061732073
:1002A0006D6F640A002025733A20666F756E6420B6
:1002B000756E616D626967756F7573206B65790A1C
:1002C00000202025733A206B6579207570203078E6
:1002D000253034580A00202025733A206B65792098
:1002E000646F776E203078253034580A002020253E
:1002F000733A206D6F642075702030782530345843
:100300000A00202025733A206D6F6420646F776E99
:10031000203078253034580A00000000001A000808
:1003200000150017001C0018000C0012000000004F
:1003300000140004611664076809620A000B000DCE
:10034000620E680F643361130005001D001B000678
:1003500000190000000000100036003700380011BE
:100360000000000000E1002C002B00015C2C002AA2
:10037000002800E50000000000000000000100016E
:100380000001000100010001000100010000000067
:100390000001000100010001000100010001000155
:1003A0000001000100010001000100010001000145
:1003B0000001000000000001000100010001000137
:1003C0000000000000010001000100010001000127
:1003D00000010001000000000044454255473A205A
:1003E00064697361626C65642E0A00444542554736
:1003F0003A20656E61626C65642E0A000A00253041
:100400003258006C65645F7461736B3A20004F6E04
:100410006573686F743A206163746976653A202564
:10042000640A000A002530313662003A2000253087
:100430003258000A722F6320303132333435363768
:1004400038394142434445460A00290A00257500CF
:100450002F002575005D280025640020002564001C
:10046000200025640020002564007C0025303258DF
:10047000006D6F7573656B6579205B62746E7C7857
:100480002079207620685D287265702F61636C2961
:100490003A205B00313A0964656C6179282A313071
:1004A0006D73293A2025750A323A09696E746572AE
:1004B00076616C286D73293A2025750A333A096DE7
:1004C00061785F73706565643A2025750A343A096E
:1004D00074696D655F746F5F6D61783A2025750A88
:1004E000353A09776865656C5F6D61785F73706533
:1004F00065643A2025750A363A09776865656C5F48
:1005000074696D655F746F5F6D61783A2025750A57
:1005100000703A097072696E742076616C7565734B
:100520000A643A097365742064656661756C747356
:100530000A75703A092B310A646E3A092D310A6C3A
:10054000743A092B31300A72743A092D31300A4558
:1005500053432F713A09717569740A0A737065659E
:1005600064203D2064656C7461202A206D61785F91
:100570007370656564202A20287265706561742037
:100580002F2074696D655F746F5F6D6178290A77DC
:10059000686572652064656C74613A206375727376
:1005A0006F723D25642C20776865656C3D25640A73
:1005B00053656520687474703A2F2F656E2E7769C5
:1005C0006B6970656469612E6F72672F77696B69FB
:1005D0002F4D6F7573655F6B6579730A004D3E2013
:1005E000004D25753A25733E20003F0A003D202529
:1005F000750A003F0A0064656661756C74730A00D1
:1006000025750A003F0A000A092D2056616C7565A0
:1006100073202D0A00710A000A092D204D6F757391
:10062000656B6579202D0A003F00433E20004C2574
:10063000640A000A092D20537461747573202D0A11
:10064000686F73745F6B6579626F6172645F6C650C
:10065000647328293A20253032580A6B6579626F15
:100660006172645F70726F746F636F6C3A202530D3
:1006700032580A6B6579626F6172645F69646C6598
:100680003A20253032580A6B65796D61705F636F6F
:100690006E6669672E6E6B726F3A20253032580A8B
:1006A00074696D65725F72656164333228293A201E
:1006B0002530386C580A000A092D20566572736976
:1006C0006F6E202D0A5649443A20307846454544FD
:1006D0002870657061736C61627329205049443AD7
:1006E00020307836303630286865786F6E33382998
:1006F000205645523A203078303030310A42554940
:100700004C443A202028466562203237203230326D
:1007100032290A4F5054494F4E533A204C554641C6
:10072000204D4F5553454B45592045585452414B48
:10073000455920434F4E534F4C4520434F4D4D415B
:100740004E44204E4B524F203531320A4743433AF4
:1007500020352E342E30204156522D4C4942433AFA
:1007600020322E302E30204156525F415243483ABB
:1007700020617672350A000A092D20436F6E736F6F
:100780006C65202D0A4553432F713A0971756974C0
:100790000A6D3A096D6F7573656B65790A000A0910
:1007A0002D204D61676963202D0A443A0944656232
:1007B0007567204D65737361676520546F67676C5B
:1007C000650A583A094D617472697820446562750A
:1007D00067204D6F646520546F67676C65202D201E
:1007E00053686F77206B65797072657373657320DA
:1007F000696E206D617472697820677269640A4B52
:100800003A094B6579626F6172642044656275676D
:1008100020546F67676C65202D2053686F77206BBD
:1008200065797072657373207265706F72740A4DAA
:100830003A094465627567204D6F75736520546F82
:1008400067676C650A563A0956657273696F6E0A76
:10085000533A095374617475730A433A09416374D6
:10086000697661746520436F6E736F6C65204D6FA0
:1008700064650A46312D4631303A0953776974630D
:100880006820746F204C6179657220302D392028E2
:10089000463130203D204C30290A302D393A095359
:1008A000776974636820746F204C617965722030B9
:1008B0002D390A47524156453A095377697463689E
:1008C00020746F204C6179657220302028616C742F
:1008D00065726E617465290A423A094A756D702025
:1008E000746F20426F6F746C6F616465720A455358
:1008F000433A094A756D7020746F20426F6F746CB3
:100900006F616465722028616C7465726E617465D4
:10091000290A453A095072696E7420454550524F74
:100920004D2053657474696E67730A425350414396
:10093000453A09436C65617220454550524F4D0A56
:100940004E3A094E4B524F20546F67676C650A0050
:100950006B65796D61705F636F6E6669672E72613A
:10096000773A20253032580A2E737761705F636FB3
:100970006E74726F6C5F636170736C6F636B3A203F
:1009800025750A2E636170736C6F636B5F746F5FA4
:10099000636F6E74726F6C3A2025750A2E737761DF
:1009A000705F6C63746C5F6C6775693A2025750ABB
:1009B0002E737761705F7263746C5F726775693AEA
:1009C0002025750A2E737761705F6C616C745F6CA3
:1009D0006775693A2025750A2E737761705F7261B9
:1009E0006C745F726775693A2025750A2E6E6F5FA9
:1009F0006775693A2025750A2E737761705F677293
:100A00006176655F6573633A2025750A2E73776199
:100A1000705F6261636B736C6173685F6261636B6B
:100A200073706163653A2025750A2E6E6B726F3A9A
:100A30002025750A0064656275675F636F6E66697D
:100A4000672E7261773A20253032580A2E656E6122
:100A5000626C653A2025750A2E6D61747269783A68
:100A60002025750A2E6B6579626F6172643A2025C4
:100A7000750A2E6D6F7573653A2025750A006565D8
:100A8000636F6E6669673A0A64656661756C745F68
:100A90006C617965723A2025750A003F004E4B5211
:100AA0004F3A206F66660A004E4B524F3A206F6EE7
:100AB0000A000A6D6F7573653A206F66660A000A50
:100AC0006D6F7573653A206F6E0A000A6B65796207
:100AD0006F6172643A206F66660A000A6B6579621C
:100AE0006F6172643A206F6E0A000A6D61747269F8
:100AF000783A206F66660A000A6D61747269783A06
:100B0000206F6E0A000A64656275673A206F666638
:100B10000A000A64656275673A206F6E0A000A0A65
:100B20004A756D70696E6720746F20626F6F746CA8
:100B30006F616465722E2E2E2000433E2000436CB0
:100B4000656172696E6720454550524F4D0A000A33
:100B5000002530325820006B6579626F6172645FE6
:100B60007265706F72743A200064656C5F6B6579B2
:100B70005F6269743A2063616E27742064656C3A21
:100B800020253032580A006164645F6B65795F62CA
:100B900069743A2063616E2774206164643A202589
:100BA0003032580A005B735D005B575D005B535D3C
:100BB000005B525D005B445D005B435D00100368B9
:100BC00000650078006F006E0033003800000014EC
:100BD00003700065007000610073006C00610062CA
:100BE00000730000000403090409025B0003010014
:100BF000A0FA09040000010301010009211101000C
:100C000001224000070581030800010904010001D9
:100C10000300000009211101000122B6000705822E
:100C20000320000109040200020300000009211151
:100C300001000122220007058303200001070503AC
:100C4000032000011201000200000008EDFE6060B8
:100C50000100010200010631FF0974A101097515A7
:100C60000026FF009520750881020976150026FFF1
:100C700000952075089102C005010902A1018502B5
:100C80000901A10005091901290815002501950888
:100C9000750181020501093009311581257F950211
:100CA0007508810609381581257F9501750881062B
:100CB000050C0A38021581257F950175088106C04B
:100CC000C005010980A101850319012AB70015019A
:100CD00026B700950175108100C0050C0901A1011E
:100CE000850419012AA002150126A002950175109C
:100CF0008100C005010906A1018506050719E02943
:100D0000E7150025019508750181020507190029DD
:100D1000EF1500250195F0750181020508190129DB
:100D200005950575019102950175039101C00501B5
:100D30000906A101050719E029E715002501950815
:100D4000750181029501750881010507190029FFC8
:100D5000150026FF00950675088100050819012970
:100D600005950575019102950175039101C0112446
:100D70001FBECFEFDAE0DEBFCDBF12E0A0E0B1E0F2
:100D8000E0EAFEE502C005900D92AC32B107D9F75A
:100D900023E0ACE2B2E001C01D92A33CB207E1F750
:100DA0000E94081C0C944E2F0C940000FF93EF93AC
:100DB000E0912C02F0912D02309709F00995EF9106
:100DC000FF910895FC018591803011F0EFDFFBCF9A
:100DD0000895FF27E0E230E247FF0CC0419597FFFE
:100DE00009C0EDE26095709580959095611D711D2B
:100DF000811D911D27FF02C0219530E350E2AA27F3
:100E0000660F771F881F991FAA1FA41710F0A41B35
:100E100063955A95A9F7AA3008F0A95FA05DAF9332
:100E2000F395611571058105910541F7ED3211F4D6
:100E3000EF93F395F21718F43F93F395FBCF8F914F
:100E4000B5DFFA95E1F70895E991F9918591803040
:100E500021F0853219F0AADFF9CF089520E0E89457
:100E600055915532C1F3503311F4689455915A336A
:100E700048F4505390F3220F022E220F220F200D20
:100E8000250FF4CF0EF4219589919991533619F3DA
:100E9000533729F1533559F1BC0188279927E89434
:100EA0005C3621F48991999168945591543639F4BE
:100EB00046EF7EF077FF0DC08FEF9FEF0AC05537EA
:100EC0004AE039F0583540E121F0523642E009F06D
:100ED0000895FF93EF937DDFEF91FF91B7CFFF93DD
:100EE000EF93FC0181918030B9F360DFFBCFFF937A
:100EF000EF9368DFF1CFDF93CF93CDB7DEB72596C1
:100F0000A3DFCF91DF9108959C01FC01E059FF4FD1
:100F100080816817A0F432974081862F90E0840F7B
:100F2000911D47FD9A956BE070E00E94D12EA901BA
:100F30006AE0869F400D511D1124CA01089580E08A
:100F400090E00895CF93DF93DC01A059BF4F4C91FF
:100F5000442391F0FC01E259FF4F80818F5F6BE0E9
:100F60000E94C32E90833396C081D1818885998554
:100F70009183808341504C93DF91CF910895EF92FC
:100F8000FF920F931F93CF93DF939C017B018C0102
:100F900000591F4FD8018C918B30B8F5F901E159F8
:100FA000FF4F811109C081E08C9312971C9210822F
:100FB00013962D933C9309C08F5FD8018C93808149
:100FC0008F5F6BE00E94C32E90838081E901BAE0BD
:100FD0008B02C00DD11D1124DE01ED92FD9285E042
:100FE000FA0101900D928A95E1F7FA0185818F83CC
:100FF00019861886D8016C91623038F0C9016250A8
:101000000E948407FC01D187C087DF91CF911F9197
:101010000F91FF90EF9008958FEF80939B03809343
:101020009C0310929D0310929F0310929E030895BB
:10103000892F8F710E94C41991E0811101C090E045
:10104000892F0895FC01948181E089270895FC018E
:101050009281DB0112968C911297981308C091E04F
:10106000238113968C91281390E0892F01C080E092
:1010700081700895EF92FF920F931F93CF93DF93A8
:10108000FC0184818823F9F07B018F01C085D18523
:101090002097C1F0BE01C8010E942708882371F083
:1010A000CE010E942208882349F0E114F10459F08E
:1010B000F70111830083D383C28305C00884D985D7
:1010C000C02DE6CF80E0DF91CF911F910F91FF906F
:1010D000EF900895CF93DF93D82FC92F892F8F7169
:1010E0000E94C41990E0FC013197E831F10590F4B9
:1010F000EA5AFF4F0C94E52E84EE10C081EE0EC02C
:1011000085EE0CC082EE0AC086EE08C083EE06C0F3
:1011100087EE04C08D2F9C2F02C080EE90E0DF91FF
:10112000CF9108959A9581159F4110F080E0089520
:1011300081E008950F931F93CF93DF938C01FC01FF
:10114000C081D181209731F0888199810E946A08FD
:1011500099838883F801C281D381209731F08881F7
:1011600099810E946A0899838883DF91CF911F91AA
:101170000F910895DC01ED91FC91309729F02081C9
:101180003181332731832083DC011296ED91FC916C
:101190001397309729F080819181992791838083DB
:1011A0000895EF92FF920F931F93CF93DF938C01DB
:1011B00060E00E9484077C01FC01C081D181CE01E6
:1011C0000E949208F70124819091E202882309F499
:1011D00045C07E01F7E0EF22FF242223F1F090FFCB
:1011E00012C0DF93CF9388E391E09F938F9382E0C7
:1011F00093E09F938F930E947B070F900F900F9027
:101200000F900F900F900E94711521E030E001C007
:10121000220FEA94EAF7822B1EC090FF12C0DF93E0
:10122000CF9388E391E09F938F938DEE92E09F930D
:101230008F930E947B070F900F900F900F900F904D
:101240000F900E94711521E030E001C0220FEA9456
:10125000EAF7209582230E94811531C02223C1F034
:1012600090FF12C0DF93CF9388E391E09F938F9319
:1012700086ED92E09F938F930E947B070F900F90D3
:101280000F900F900F900F90CE010E94F60A17C09A
:1012900090FF12C0DF93CF9388E391E09F938F93E9
:1012A00081EC92E09F938F930E947B070F900F90A9
:1012B0000F900F900F900F90CE010E940C0BC80161
:1012C000DF91CF911F910F91FF90EF900C94A207A7
:1012D000AF92BF92CF92DF92EF92FF920F931F9344
:1012E000CF93DF9300D000D0CDB7DEB76C0160E0C4
:1012F0000E9484077C01FC01808191810E94180872
:10130000811117C08091E20280FF0EC08DE291E052
:101310009F938F9385EA92E09F938F930E947B0720
:101320000F900F900F900F90C6010E94D10811E00E
:101330008EC0F701808191810E941808882309F1ED
:10134000C7010E942208182F8823D9F08091E20259
:1013500080FF0EC08DE291E09F938F9385E892E02D
:101360009F938F930E947B070F900F900F900F9089
:101370001A821982FC82EB82CE0101960E949A08A1
:101380001FC0BE016F5F7F4FC7010E943A08182F30
:101390008823D1F08091E20280FF0EC08DE291E0BF
:1013A0009F938F9380E592E09F938F930E947B079A
:1013B0000F900F900F900F90CE0101960E94BA08E7
:1013C000C6010E94D10843C0F701A084B184A114D2
:1013D000B10449F160E070E0C5010E943A08082FAD
:1013E0008823F9F08091E20280FF0EC08DE291E047
:1013F0009F938F9383E192E09F938F930E947B074B
:101400000F900F900F900F90FA82E9821C821B823E
:10141000CE0101960E949A08C6010E94D108102FA1
:1014200016C0F501D2CF8091E20280FF0FC08DE29D
:1014300091E09F938F9384EF91E09F938F930E940D
:101440007B070F900F900F900F9001C010E0812F3D
:101450000F900F900F900F90DF91CF911F910F91F0
:10146000FF90EF90DF90CF90BF90AF900895EF92F4
:10147000FF920F931F93CF93DF9381302CE5920758
:1014800011F4C1E075C08B01EC0180919D038111C5
:101490001AC0CE010E941808811115C08091E20285
:1014A000C82FC17080FFEDCF89E191E09F938F93AA
:1014B00080EE91E09F938F930E947B070F900F9097
:1014C0000F900F9055C08091E20280FF0EC089E11D
:1014D00091E09F938F9389EC91E09F938F930E946B
:1014E0007B070F900F900F900F90A801BE018DE227
:1014F00093E00E94BF0709E111E089EAE82E81E04C
:10150000F82E80919D038823E9F09091E20290FFEC
:101510000EC01F928F931F930F93FF92EF920E9422
:101520007B070F900F900F900F900F900F908DE210
:1015300093E00E946809C82F8111E3CF8091E202F5
:1015400080FD02C0C0E014C080919D031F928F9364
:1015500089E191E09F938F9386E891E09F938F9329
:101560000E947B070F900F900F900F900F900F909D
:101570008C2FDF91CF911F910F91FF90EF900895E5
:101580009C013A9521153F4130F5BC0166277270E8
:10159000AC01442754709C012227387094FF0FC07F
:1015A00090FF02C080E101C080E0672B09F08062FB
:1015B000452B09F08064232B79F080680895892FEA
:1015C0008170672B09F08260452B09F08460232B22
:1015D00019F08860089580E00895CF93DF93EB01C0
:1015E0000E94C00AFE01DF91CF910994CF93DF934F
:1015F000EC01805E9109089710F0209719F46DE6D0
:101600007DE002C068EF7FE0CE010E94ED0A8C2FE2
:10161000DF91CF910C94BE0CCF93DF93EC010E942D
:10162000190DCE01805E9109089710F0209719F4EA
:1016300064E77DE002C06FEF7FE0CE01DF91CF91E4
:101640000C94ED0A81E008950C94370A08950C94E7
:10165000260B1F93CF93DF9300D000D01F92CDB7FE
:10166000DEB749835A836B8330912F0289819A8137
:10167000311114C0662359F0222349F00E94CB1186
:10168000182F682F89819A810E94741103C00E94CB
:101690009F11182F69817A81812F04C00E94CB117C
:1016A00069817A810F900F900F900F900F90DF91CA
:1016B000CF911F910C941819FC01262F4081518164
:1016C0006281738184810C94290B81E00895CF930A
:1016D000DF93EC0160E00E945C0BBE01DF91CF91D3
:1016E0000C94270B0C94A01A0C949E1A08950E9437
:1016F0001E100E94760B2FEF84E39CE02150804067
:101700009040E1F700C000000C94E7260F931F9370
:10171000CF93DF938C0161E00E945C0BEC01B80178
:101720000E94240B882309F45BC0B801CE010E94FB
:101730002724882309F454C0B801CE010E94201F39
:10174000882309F44DC0B801CE010E948323882369
:1017500009F446C0F80182818823D9F1CF3D8CE598
:10176000D80779F140F4C115FCE5DF0791F0C130ED
:10177000DC4591F02EC0CC35EDE5DE0741F1CD35ED
:10178000FDE5DF0709F1CB35DD4519F50E9465164A
:1017900020C00E94770B24C08091E202C82FC09520
:1017A000C170C0FB80F98093E202CC2329F08BEE5C
:1017B00093E00E94E20614C089ED93E00E94E206E5
:1017C00010C00E9419170CC00E945C1602C00E9433
:1017D0006816C801DF91CF911F910F910C94220BD5
:1017E000C0E08C2FDF91CF911F910F9108950E943F
:1017F0001B260C94350C0E94380C0C9421268295E3
:10180000982F937344E0949F900111248C7C8695CB
:101810008695282B822F8575880F2A7A2695822B0C
:101820000895CF93DF93D92F0E94FF0BC82F8D2FE0
:101830000E94FF0B2C2F30E0322F2227A901482BCA
:10184000CA01DF91CF91089508950C94240C81E092
:1018500008950C94270C0895CF93C82F0E94250C4F
:101860008C2F0E94290CCF91089580E00C942C0CB1
:101870000E9483240C942C0CCF930E948324C82FA5
:1018800080912E02C81741F1C0932E028091E2028E
:1018900082FF1EC080FF04C083E094E00E94E20645
:1018A0008091E20280FF0CC01F92CF938EEF93E0F5
:1018B0009F938F930E947B070F900F900F900F9034
:1018C0008091E20280FF04C08CEF93E00E94E20668
:1018D0008C2FCF910C942C0CCF910895CF93DF9344
:1018E000CDB7DEB72B970FB6F894DEBF0FBECDBFD6
:1018F0004F83588769877A878B8761110E94941577
:101900009E012F5F3F4F86E0F90111928A95E9F71A
:1019100085E0FE013796D90101900D928A95E1F795
:1019200089819A814C815D81452B31F09F3F31F453
:1019300091E08F3F19F403C091E001C090E090FF67
:1019400009C049815A816B817C818D819E810E9471
:10195000B21405C0C9010E94650B8111F2CF2B960C
:101960000FB6F894DEBF0FBECDBFDF91CF910895C3
:10197000FC01808191810E940D120895CF938823EC
:1019800009F455C0C82F8CEF8C0F813AF8F48C2FD6
:101990000E942C2381114BC06C2F809102019091E9
:1019A00003010E943425882349F06C2F80910201A5
:1019B000909103010E94E1250E94B6156C2F809141
:1019C0000201909103010E94D6250CC080E28C0F89
:1019D000883058F4C77081E001C0880FCA95EAF7D3
:1019E0000E947415CF910C94B615EBE5EC0FE33023
:1019F00040F4F0E0E558FE4F808190E0CF910C94E8
:101A0000F224E8E5EC0FE73150F4F0E0EE0FFF1FB1
:101A1000E35BFE4F80819181CF910C940825CD3EF0
:101A200030F08C2F0E948D1CCF910C945F1DCF91B4
:101A30000895882389F19CEF980F913A40F4682F1C
:101A400080910201909103010E94E1250DC090E276
:101A5000980F983058F4877091E001C0990F8A95DB
:101A6000EAF7892F0E947A150C94B6159BE5980F1A
:101A7000933020F480E090E00C94F22498E5980FE5
:101A8000973120F480E090E00C9408258D3E20F002
:101A90000E94E81C0C945F1D08951F93CF93DF9361
:101AA000182FEB010E94BE0C209741F08FE99FE0B8
:101AB0000197F1F700C000002197F6CF812FDF9149
:101AC000CF911F910C94190D893319F060E070E0EB
:101AD00002C060E570E00C944D0D882321F00E9457
:101AE00074150C94B6150895882321F00E947A1578
:101AF0000C94B6150895CF92DF92EF92FF920F9358
:101B00001F93CF93DF937C01D62FC72FFC01128147
:101B1000058102950F700E946A158823B9F0112380
:101B2000A9F08C2F807F803421F080E28D0F8830E7
:101B300068F08091A10382FD09C082E00E94161620
:101B40000E946A1591E0D82ED92601C0D12CCC2E46
:101B5000C2948FE0C8228C2D90E08C30910508F063
:101B6000CFC1FC01E259FF4F0C94E52E8C2F807FF2
:101B7000CF70882311F0C295C07F112399F0CC2338
:101B800009F4AAC180E28D0F883010F0D11104C091
:101B90008C2F0E94741503C08C2F0E9487150E9401
:101BA000B6159AC18D2F0E94190DCC2309F4A8C136
:101BB00080E28D0F883038F1DD2329F18C2F0E94CF
:101BC0008D1524C08C2F807FCF70803211F0C2958C
:101BD000C07FDD2319F0D130A1F13DC08091A10378
:101BE00082FF17C0112349F0CC2329F08C2F0E94CB
:101BF00074150E94B61580E070C180E00E94190D36
:101C0000CC2309F47DC18C2F0E947A150E94B61551
:101C100077C1112371F0002341F0013031F40E94AB
:101C200097158C2B0E949F156BC10E9497158C2BCA
:101C30001DC0002319F0013009F462C10E94AC15E7
:101C400025C0112321F0063008F05AC10EC005301E
:101C500008F056C11BC0112361F0002331F0F701D9
:101C6000858180FF39C18F7085838C2F0E946D0D17
:101C700047C1002359F0D93309F03FC1FFEF07EE08
:101C800013E0F15000401040E1F735C18C2F0E9465
:101C9000740D36C18C2F86958695837019F081302E
:101CA00061F02EC1112321F08D2F9C2F937002C063
:101CB00080E090E00E94F2242BC1112321F08D2FAF
:101CC0009C2F937002C080E090E00E94082520C104
:101CD0008D2F112319F00E948D1C02C00E94E81C58
:101CE0000E945F1D15C18C2F837009F047C0111130
:101CF0000BC12D2F229526952770220F220F6D2FB5
:101D00006F70862F90E0A0E0B0E0022E04C0880F34
:101D1000991FAA1FBB1F0A94D2F7D4FF10C04FE02F
:101D200050E060E070E004C0440F551F661F771F4D
:101D30002A95D2F7409550956095709503C040E084
:101D400050E0BA01C695C695C3708A019B01082B65
:101D5000192B2A2B3B2BC901B801C23049F058F48A
:101D6000C13019F00E948A10CFC00E947810CCC0F8
:101D70000E949C10C9C00E947610C6C0112319F0A1
:101D80008C2F817001C08695882309F4BDC02D2F4A
:101D9000229526952770220F220F6D2F6F70862FA8
:101DA00090E0A0E0B0E0022E04C0880F991FAA1FA7
:101DB000BB1F0A94D2F7D4FF10C04FE050E060E0A0
:101DC00070E004C0440F551F661F771F2A95D2F795
:101DD000409550956095709503C040E050E0BA0181
:101DE000C695C695C3708A019B01082B192B2A2B17
:101DF0003B2BC901B801C23049F058F4C13019F089
:101E00000E944F1181C00E943D117EC00E9461114D
:101E10007BC00E94B01078C0CF70112339F08C2F96
:101E20000E94D6108D2F0E946D0D6EC08D2F0E94C6
:101E3000740D8C2F0E94F71067C0D23F21F128F457
:101E4000D03F41F0D13FC1F043C0D33F19F1D43F5F
:101E500079F03EC0112341F0053008F051C08C2FBD
:101E60008F710E941C114CC0063008F049C0F7CF9A
:101E70008091A10382FF18C0112339F08C2F8F713C
:101E80000E94D6103DC01123C9F38C2F8F710E9480
:101E9000F71036C0112329F08C2F8F710E94C110CA
:101EA0002FC00E94BC102CC0112349F0CF718C2F81
:101EB0000E94D61063E08C2F0E94FB1521C081E0A8
:101EC0000E9416160230E0F082E00E94161618C03A
:101ED000112331F0002391F28D2F0E94BE0C10C00F
:101EE000002399F2D93349F41FEF27EE33E0115064
:101EF00020403040E1F700C000008D2F0E94190DF6
:101F000088EF8C0D843020F40E9483240E942C0CD6
:101F1000DD20C9F00E94661580FD15C0F701128210
:101F20000E9460150E94D610C7010E94C40F0E9433
:101F30006015DF91CF911F910F91FF90EF90DF908F
:101F4000CF900C94F710DF91CF911F910F91FF90DC
:101F5000EF90DF90CF9008950F931F93CF93DF936F
:101F6000EC01688179818A810E9418128C010E949B
:101F700073110E946410B801CE010E947B0DDF91A5
:101F8000CF911F910F910895CF93DF93EC0198812A
:101F900089812B813C81232B31F08F3F31F481E00B
:101FA0009F3F19F403C081E001C080E080FD1DC0A7
:101FB000CE010E94860B811110C00E946A158823F1
:101FC000A1F08A81882389F08091A10382FD0DC050
:101FD00082E0DF91CF910C941616CE010E94AC0FD7
:101FE000CE01DF91CF910C94670BDF91CF910895D3
:101FF000882321F00E9487150C94B6150895882334
:1020000021F00E948D150C94B615089580E090E0A3
:102010000E94F22480E090E00E9408250E9494151E
:102020000E94B6150E94121F0C945F1D8091020140
:10203000909103010E94EC250C9406100E948415D7
:102040000C94161092959F70963079F010F492507F
:1020500001C09A50923068F4803F69F018F4883ECD
:1020600040F409C0843F29F406C0883E20F0813F37
:1020700011F080E0089581E00895FC018081918154
:102080000E940D120E9422100895CF93DF9300D07A
:1020900000D01F92CDB7DEB70F900F900F900F902A
:1020A0000F90DF91CF910895CF93DF9300D000D0B0
:1020B00000D0CDB7DEB726960FB6F894DEBF0FBEC0
:1020C000CDBFDF91CF910895089508950C946510C8
:1020D0000C9466100E946810609352027093530231
:1020E00080935402909355020C9406100C946A103D
:1020F0000F931F93009152021091530220915402AA
:1021000030915502602B712B822B932B1F910F91D5
:102110000C946A100F931F93009152021091530276
:10212000209154023091550260237123822393231E
:102130001F910F910C946A100F931F9300915202FC
:10214000109153022091540230915502602771275B
:10215000822793271F910F910C946A100C9465109D
:102160000E94AE1060934E0270934F028093500213
:10217000909351020C94061060E070E0CB010C9437
:10218000B0100F931F9341E050E060E070E08A01CF
:102190009B0104C0000F111F221F331F8A95D2F725
:1021A000C901B8011F910F910C94B0100F931F93A8
:1021B00041E050E060E070E004C0440F551F661F2E
:1021C000771F8A95D2F780914E0290914F02A0918D
:1021D0005002B09151028A019B01082B192B2A2B26
:1021E0003B2BC901B8011F910F910C94B0100F93B4
:1021F0001F9341E050E060E070E004C0440F551FC1
:10220000661F771F8A95D2F7409550956095709517
:1022100080914E0290914F02A0915002B0915102D4
:102220008A019B01082319232A233B23C901B801F2
:102230001F910F910C94B0100F931F9341E050E049
:1022400060E070E004C0440F551F661F771F8A9539
:10225000D2F780914E0290914F02A0915002B0911E
:1022600051028A019B01082719272A273B27C90108
:10227000B8011F910F910C94B0100F931F93009110
:102280004E0210914F022091500230915102602B6A
:10229000712B822B932B1F910F910C94B0100F93E5
:1022A0001F9300914E0210914F02209150023091E5
:1022B000510260237123822393231F910F910C9469
:1022C000B0100F931F9300914E0210914F02209176
:1022D00050023091510260277127822793271F9166
:1022E0000F910C94B01008952CE0929F800D112452
:1022F000E82FE695E695E695877051E001C0550F09
:102300008A95EAF785E0E89FF0011124E05DFD4F32
:1023100020E030E070E04081CB01022E02C09695B3
:1023200087950A94E2F78170819584278523842715
:1023300081932F5F3F4F2530310569F708952CE0D9
:10234000929F800D1124682F669566956695982F4B
:10235000977085E0689FB001112440E050E080E074
:10236000FB01E40FF51FE05DFD4F208130E0092EF9
:1023700002C0369527950A94E2F721703327042E80
:1023800001C0220F0A94EAF7822B4F5F5F4F45305E
:10239000510531F70895BF92CF92DF92EF92FF92ED
:1023A0000F931F93CF93DF938C01C0904E02D09078
:1023B0004F02E0905002F0905102809152029091B1
:1023C0005302A0915402B0915502C82AD92AEA2A90
:1023D000FB2ACFE1D0E0D701C6010C2E04C0B69590
:1023E000A795979587950A94D2F780FD04C0219709
:1023F00090F7B12C07C0BC2EB8018C2F0E942B196E
:102400000197A9F38B2DDF91CF911F910F91FF9031
:10241000EF90DF90CF90BF900895CF93DF93EC01C2
:102420000E94CB11BE010E942B19DF91CF9108951C
:102430001F93CF93DF93EB0190912F02992321F00B
:10244000CB010E940D1213C0882349F0CB010E94DA
:10245000CB11182F682FCE010E94741104C0CB013C
:102460000E949F11182FBE01812F0E942B19DF910E
:10247000CF911F9108951F93CF93DF93C091560280
:1024800016E080915702C81799F0D0E01C9FF00128
:102490001D9FF00D1124E85AFD4F4081518162814A
:1024A0007381848195810E9454102196C770E9CF71
:1024B000DF91CF911F910895409188025091890238
:1024C00060918A0270918B0280918C0290918D02B2
:1024D0000C945410EF92FF920F931F93CF93DF93BE
:1024E00080918D0282958F7009F065C080918A027B
:1024F000882309F460C080915602F0905702109131
:1025000088020091890260918B0270918C0291E0A7
:102510001F3F09F090E0C0910001D0910101292FE7
:1025200096E0E92E8F1509F446C06115710521F07A
:102530000F3F21F030E003C031E001C0322F90E0C6
:1025400030FD36C0E89EF001E99EF00D1124DF0158
:10255000A85ABD4F11963C911197301329C03C9158
:10256000311326C012963C911297311121C0139657
:102570004D915C911497461B570B4C175D07C0F4A7
:1025800080918D028F70806180938D02E35AFD4FA0
:1025900080818F708061808388E892E00E94C40F00
:1025A000DF91CF911F910F91FF90EF900C943B1210
:1025B00001968770B7CFDF91CF911F910F91FF9058
:1025C000EF9008959F92AF92BF92CF92DF92EF92D9
:1025D000FF920F931F93CF93DF93CDB7DEB7619731
:1025E0000FB6F894DEBF0FBECDBF8C0185E0F801B9
:1025F000DE011D9601900D928A95E1F7D8011296A1
:10260000EC9090918802E091890220918B023091A8
:102610008C022115310531F0EF3F31F481E09F3F0D
:1026200019F403C081E001C080E0B82FB1709B2E87
:1026300080FD47C1D8014C9111965C91119713967A
:10264000AD90BC90149788E8C82E82E0D82EF09008
:102650008A02B501621B730B2091000130910101C8
:10266000FF2009F4D9C080918D026217730708F02A
:1026700095C0282F207F09F052C05E1313C0491364
:1026800011C0FE2CE1100EC08F70806180938D020E
:102690000E945C12C6010E94C40F80918D02F80155
:1026A00085834DC1AB2831F05F3F31F481E04F3F6E
:1026B00019F403C081E001C080E080FD03C081E027
:1026C0008E2502C080E090E0F82FF170FF2E80FF91
:1026D0001CC0809156022091570236E0821709F4FF
:1026E0000BC190E0389FF001399FF00D1124E85A9A
:1026F000FD4F6181561306C06081461303C062819D
:10270000E61203C001968770E9CFFE2CEE2009F493
:1027100016C180918D02816080938D0254C05E133A
:1027200006C0491304C0E11002C0F80199C0C801F5
:102730000E943D10882361F1EE2051F120918D021D
:10274000822F82958F7090E0029774F080918802BA
:102750009091890298878F831986BB86AA862C87D9
:10276000CE0107960E94C40F86E0F801A8E8B2E007
:1027700001900D928A95E1F70E946A120E945C1204
:102780000AC05E1711F1C8010E943D1081112CC0D2
:10279000C8010E94C40FFF24F394D1C0282F207FCA
:1027A00081F77A2DB98AA88A6E2D89890E944510F1
:1027B00088E892E00E94C40F86E0D6011D928A95B7
:1027C000E9F70E945C12F12CBAC04913DCCFE1108A
:1027D000DACFF8018583C8010E94C40F86E0D601D4
:1027E0001D928A95E9F7ABC0EE2091F220918D02FF
:1027F000822F82958F7090E002970CF4B5CF809174
:102800008802909189029A8389831B82BD82AC825F
:102810002E83CE010196A6CF6217730708F044C03D
:10282000FE2CEE2009F4B4CF5E1330C049132EC045
:1028300020918D0220FD21C0822F82958F70482F1C
:1028400050E041155105C9F0F80125834F3051057D
:1028500041F08F5F982F9295907F822F8F70892BF8
:102860008583C8010E94C40F86E0F801A8E8B2E0A1
:1028700001900D928A95E1F73CC086E0F801A8E846
:10288000B2E001900D928A95E1F759C0C8010E940B
:102890003D10811169CF80918D02816080938D02FE
:1028A000C8010E94C40F4BC07A2DB98AA88A6E2D28
:1028B00089890E94451086E0D6011D928A95E9F724
:1028C00018C0EE2009F464CFC8010E943D10F82E14
:1028D000882309F45DCF86E0F801A8E8B2E0019012
:1028E0000D928A95E1F788E892E00E94B80C0E9468
:1028F0006A120E945C1223C04D875E878D859E857B
:102900000E940D12292F22952F70223028F49F70DB
:1029100039F0811105C00BC0243028F49F7049F4B0
:10292000805E883020F0C8010E94C40F9F2CF92CD3
:1029300006C0D80115969C91907F91F7F8CF8F2D06
:1029400061960FB6F894DEBF0FBECDBFDF91CF9179
:102950001F910F91FF90EF90DF90CF90BF90AF90BD
:102960009F9008951F93CF93DF93CDB7DEB72C9739
:102970000FB6F894DEBF0FBECDBF4F83588769876F
:102980007A878B879C87CE0107960E94E212882364
:10299000D1F09F8188852A853B85232B31F08F3F9D
:1029A00031F481E09F3F19F403C081E001C080E071
:1029B00080FD47C04F81588569857A858B859C85C8
:1029C0000E9454103EC086E0FE013796DE0111964B
:1029D00001900D928A95E1F7FF81E8856A857B85F4
:1029E0006115710531F0EF3F31F481E0FF3F19F4DB
:1029F00003C081E001C080E080FD23C02091570228
:102A000030E0C9010196877099274091560250E045
:102A100084179507F1F1F983EA837D836C8396E04F
:102A2000929FD001939FB00D1124A85ABD4FFE0173
:102A3000319601900D929A95E1F7809357020E948A
:102A40003B1216E08091560290915702891771F15E
:102A5000189FC0011124885A9D4F0E94E2128823BA
:102A600029F1E09156021E9FF0011124E85AFD4F12
:102A70004081518162817381848195810E945410CB
:102A80008091560290E001968770992780935602B4
:102A9000D9CF0E941E101092570210925602E8E8F9
:102AA000F2E086E0DF011D928A95E9F72C960FB6D9
:102AB000F894DEBF0FBECDBFDF91CF911F91089577
:102AC0008091AE0285958595859508958091AE0299
:102AD000877008959091AE02977081E009F480E0CC
:102AE00008958091D10208959091D102892B80930D
:102AF000D102089580959091D10289238093D102CB
:102B000008958093D10208951092D1020895909172
:102B1000D002892B8093D002089580959091D002A5
:102B200089238093D00208951092D0020895809155
:102B3000AF02089508950C949A150C949B159091EA
:102B4000A10392FD08C09091AF02981721F08093E5
:102B5000AF020C949D1508958091AF02882329F04F
:102B60001092AF0280E00C949D150895CF93DF93EF
:102B7000E0910201F09103018091D1028083E09104
:102B80000201F091030190818091D002892B808312
:102B90008091AF02882381F0E0910201F09103015E
:102BA0009081892B808380910201909103010E9482
:102BB0001E2581110E94AC15C0910201D091030124
:102BC00040E250E06EE872E0CE010E94FF2E892BB9
:102BD00069F080E2FE01AEE8B2E001900D928A95C4
:102BE000E1F7CE01DF91CF910C948F24DF91CF914B
:102BF00008950C949A159091A10392FD10C098E04D
:102C0000899F90011124262B2093AE020E94D6109A
:102C10008091AE028595859585950C94F9150C9457
:102C2000D6101092AE0280E00C94F9152091AE02FD
:102C3000809582238093AE02982F977099F430E0AC
:102C4000482F082E000C550B2417350759F090918A
:102C5000A10392FD07C08595859585950E94F71083
:102C60000C9411160895CF939091A10392FB222703
:102C700020F92817F9F0C82F892FC0FB82F980931B
:102C8000A1038091A0039091A1030E94951682E078
:102C90000E9416168091E20280FF0CC01F92CF9313
:102CA0008EE094E09F938F930E947B070F900F908C
:102CB0000F900F90CF9108958091A10382FB8827F8
:102CC00080F991E089270C94331681E00C94331637
:102CD00080E00C9433166FEF7FEF80E090E00C946F
:102CE000382F80E090E00E94142F21E0893E9E4F13
:102CF00009F020E0822F089582E090E00C940C2FE0
:102D000083E090E00C940C2FCF9384E090E00E943D
:102D10000C2FC82F82E290E00E940C2F2C2F30E065
:102D2000A901582BCA01CF910895CF93C92F682FBD
:102D300084E090E00E941A2F6C2F82E290E0CF9105
:102D40000C941A2FAB01BC018FE090E00C942C2F57
:102D5000AB01BC0183E190E00C942C2F60E070E0AB
:102D6000CB010C94A81660E070E0CB010E94A21683
:102D70000C94AE1669EE7EEF80E090E00E94382F52
:102D800060E082E090E00E941A2F60E083E090E033
:102D90000E941A2F10925202109253021092540263
:102DA0001092550260E084E090E00E941A2F60E0EB
:102DB00082E290E00E941A2F60E085E090E00E949D
:102DC0001A2F60E086E090E00E941A2F6FEF87E0F4
:102DD00090E00E941A2F40E050E0BA0188E090E0B5
:102DE0000E942C2F60E08DE090E00E941A2F40E0BE
:102DF00050E0BA0188E190E00E942C2F60E087E16A
:102E000090E00E941A2F40E050E0BA018CE190E07F
:102E10000E942C2F60E070E080E290E00E94382F4A
:102E200040E050E0BA0188E190E00E942C2F0C9421
:102E3000B3160C94BA16682F8EE090E00C941A2FFB
:102E40000E94A6266093DE027093DF028093E00268
:102E50009093E1026093DA027093DB028093DC02CC
:102E60009093DD02089585B7806885BF85B7806837
:102E700085BF089581E008950C943A1708950C9445
:102E80003E170C943E170C9441170C943E170C946B
:102E900045170C943E170E94331781E099E20E9477
:102EA00079240E9449170C9447170E943F170C94ED
:102EB0003E170E941F1A0C942B0C0E9491260E9410
:102EC000571B0E9459170C9443175F926F927F9281
:102ED0008F929F92AF92BF92CF92DF92EF92FF922A
:102EE0000F931F93CF93DF93CDB7DEB72A970FB61B
:102EF000F894DEBF0FBECDBF0E946C1BC82E81119F
:102F00000E94201732ED832E32E0932E00E010E075
:102F1000502E802F0E94431A5C01F4016190719041
:102F20004F016826792661147104B1F40F5F1F4FB9
:102F30000430110569F78FEF89838A831B820E9411
:102F40009A268160782F9D838C8349815A816B8179
:102F50008D810E946E0C3AC08091E20281FD0E9438
:102F60004C1AD12CEE24E394F12CC3018E219F2125
:102F7000892B29F10E943C178823A9F0DE825F8209
:102F8000AE20BF2081E0AB2809F480E088870E9452
:102F90009A268160782F9A8789874E815F8168851C
:102FA0008A850E946E0C000F111FF801EE52FD4F32
:102FB00080819181E826F926F182E08207C0D394CE
:102FC000EE0CFF1CFCE0DF12D0CFB0CF81E0C110CF
:102FD00001C080E02A960FB6F894DEBF0FBECDBFC9
:102FE000DF91CF911F910F91FF90EF90DF90CF90E5
:102FF000BF90AF909F908F907F906F905F9008955B
:103000000E9465170E94FF1D0C943C0CCF93DF9328
:103010000E943019EC01811521E5920708F045C0A6
:10302000811530E5930708F094C0883E910528F596
:10303000803E910508F0F8C0883A910570F4853A11
:10304000910508F07CC08130910509F475C008F441
:10305000E8C0049708F0E8C0E4C08F3B910508F091
:10306000E0C0C85AD0E0CC0FDD1FC258DE4F099037
:10307000D881C02DCE019464D8C0811540E2940758
:1030800058F4811551E0950708F0CEC08D3E9105AA
:1030900008F4C7C09065C9C0C11580E4D80708F41A
:1030A000C0C0DF70CE01906AC0C0811525E59207CF
:1030B000A8F4811534E5930708F095C0811543E520
:1030C000940708F07BC0811552E5950708F061C0B0
:1030D000D82FCC27CE01816F906AA7C0C11589E592
:1030E000D807A0F4C11528E5D20708F082C0C115A1
:1030F00036E5D30708F095C08C2F0E94C4198F7154
:1031000090E0D82FCC27CE0190628FC0C1154AE540
:10311000D40708F474C0CE0190568115904208F08F
:1031200080C08D2F8F710E94C419DD27D0628F71EE
:10313000AE01582BCA0179C081E090E076C0C55A33
:10314000D0E0C455DE4F8881C82FD0E0CE01906416
:103150006CC074E0969587957A95E1F7282F2370D7
:103160003C2F337081E090E002C0880F991F3A95A0
:10317000E2F79C68AC01522B9A019C2F9F709695A8
:10318000969550E2959FE0011124C9018C2B9D2B4F
:103190004CC08370992721E030E002C0220F331F1A
:1031A0008A95E2F79C2F9695969580E2989FE0018C
:1031B0001124C22BD32BCE019C6837C08370992772
:1031C00021E030E002C0220F331F8A95E2F79C2FE6
:1031D0009695969540E2949FE0011124C22BD32B43
:1031E000CE019A6822C0D82FCC27CE01846F906A76
:1031F0001CC0DC2FCC27CE01806F906A16C08C2FAC
:103200008F700E94C41994E0D695C7959A95E1F7FE
:10321000CF70D0E0DC2FCC27D0699E01282BC901CC
:1032200004C080E090E001C0CE01DF91CF9108950D
:1032300020E3829FC0011124FC012CE0729FE00D6D
:10324000F11D1124E60FF11DEE0FFF1FE75EFC4F8D
:103250008591949108950E9418190E940618089566
:103260008238910569F1B0F48133910509F46DC09C
:1032700048F48932910509F463C08A32910509F452
:1032800069C008958533910509F455C089339105C6
:10329000B9F00895833E910569F138F4803E9105B7
:1032A000B1F0823E910509F10895863E9105A9F19C
:1032B000873E9105B9F1843E910509F064C023C0B1
:1032C0002091A00320FD4FC021FD4DC008958091A5
:1032D000A00380FD44C08091A10380FF44C0809181
:1032E000A00384FD42C083EE4DC08091A00382FF05
:1032F00038C0F5CF8091A00382FD33C08091A10337
:1033000080FD31C0ECCF8091A10381FF32C080915C
:10331000A00384FD2AC087EE35C08091A00383FFFF
:1033200026C0F5CF8091A00383FD21C08091A10329
:1033300081FD1FC0ECCF8091A00385FD1CC01DC086
:103340008091A00385FD19C016C08091A00386FD61
:1033500016C017C08091A00386FD13C010C089E37A
:1033600011C082EE0FC080EE0DC080E00BC086EE73
:1033700009C084EE07C089E205C085E303C08AE284
:1033800001C081E390E008959091A00392FF0DC0E9
:10339000282F2871283019F4877F846006C0282FD1
:1033A0002471243011F48B7F886093FF0DC0282F87
:1033B0002871283119F4877E846106C0282F247172
:1033C000243111F48B7E88612091A10320FF0DC070
:1033D000382F3871383019F4877F816006C0382F54
:1033E0003171313011F48E7F886021FF0DC0282F9C
:1033F0002871283119F4877E816106C0282F217138
:10340000213111F48E7E886194FD877E08950C949D
:103410006B160E946C1B8FE39CE90197F1F700C0CB
:1034200000000E946C1B80E00E94431A80FF04C0D1
:103430000E94071A0C94E72608950C94091A0E941A
:103440007116811102C00E9419170E947C16809388
:10345000E2020E9484169093A1038093A0030E942D
:103460001D1A0E948016682F70E080E090E00E9494
:10347000761060914E0270914F02809150029091AF
:1034800051020C94AE10E82FF0E0EE0FFF1FE6554E
:10349000FC4F808191810895CF92DF92EF92FF924D
:1034A0000F931F93CF93DF9383E394E00E94E20690
:1034B0008AEAE82E83E0F82EC0E0D0E09EE2C92E32
:1034C00094E0D92E05E214E0DF93CF93DF92CF9200
:1034D0000E947B078BE294E00E94E206F701819153
:1034E00091917F010E94110C9F938F931F930F93D3
:1034F0000E947B0783E294E00E94E20621968DB74A
:103500009EB708960FB6F8949EBF0FBE8DBFC4300D
:10351000D105D1F6DF91CF911F910F91FF90EF90E0
:10352000DF90CF90089580EA8A95F1F7089500C062
:1035300008950C94931A08950C949B1A0C949C1A59
:103540000C940C08F894E82FE295EF70F0E031A1AC
:10355000282F2F7081E090E001C0880F2A95EAF7AC
:10356000982F9095932391A392A1892B82A378946D
:1035700008950F931F93CF93DF93CFEAD1E0899102
:103580008F3F11F00E94A21A81E0CB3BD807B9F718
:10359000CBEBD1E00FEB11E089918F3F11F00E944E
:1035A000A21A0C171D07C1F7DF91CF911F910F9140
:1035B0000895AF92BF92DF92EF92FF920F931F9305
:1035C000CF93DF93C62FD0E0C155DE4F28812F3F28
:1035D00009F463C08A01F62EE92ED82EF894E22F62
:1035E000E295EF70F0E091A1822F8F7021E030E042
:1035F00001C0220F8A95EAF7892F822B81A382A12D
:103600002095282322A378940E94971A8BEBA82E4A
:1036100081E0B82EED2DFE2D9F01285F3F4FE12C5C
:10362000A80140955095D5016D915D016F3FC9F09E
:10363000862F82958F7090E0DC0190968C9190E0BF
:103640006F7002C0959587956A95E2F780FD09C075
:1036500080819181802B912B91838083EE24E39450
:1036600006C0808191818423952391838083329643
:10367000E217F307C1F688818F3F11F00E94A21A6A
:103680006E2D8F2DDF91CF911F910F91FF90EF90B5
:10369000DF90BF90AF900C94991ADF91CF911F915A
:1036A0000F91FF90EF90DF90BF90AF9008950E9430
:1036B000B91A88E0EAEAF3E0DF01982F1D929A95A3
:1036C000E9F7E2EAF3E0DF011D928A95E9F784E089
:1036D0000E94C11B0C94720BCF92DF92FF920F934A
:1036E0001F93CF93DF93CDB7DEB728970FB6F8942B
:1036F000DEBF0FBECDBF8E010F5F1F4F88E0F80108
:1037000011928A95E9F7F12CCC24C394D12CA6010F
:103710006F2DC8010E94D91AF394CC0CDD1CFCE07B
:10372000FF12F5CF48E050E0B80182EA93E00E9432
:10373000FF2EFF24F394009709F4F12C892B41F01C
:1037400088E0F801A2EAB3E001900D928A95E1F7D2
:103750002F2D44E06AEA73E082EA93E00E94C21BE4
:103760000E94740B8F2D28960FB6F894DEBF0FBE03
:10377000CDBFDF91CF911F910F91FF90DF90CF9040
:1037800008950895FF920F931F93CF93DF93F82E20
:10379000092F162FD72FC42F222349F081E08093C1
:1037A000E5020E949A269093E4028093E3028091BE
:1037B000E5028823D9F08091E3029091E4020E940F
:1037C000B226059798F0EF2DF02FA12FBD2F80E0A6
:1037D00090E04C2F50E08417950734F421913191FB
:1037E0002D933D930196F7CF1092E502DF91CF9193
:1037F0001F910F91FF9008950E947D290E945D17EF
:103800000C9489290E948D290E9400180C94AB29E0
:103810000E9438260E9464290E944B170E94FC1BBC
:103820000E94021C0E945517FBCF8091EC0280FF82
:1038300006C06091090170E0660F771F26C081FF06
:1038400004C06091090184E005C082FF07C0609157
:10385000090188E0689FB001112417C09091EB0224
:103860009923D1F060910801961788F720910901FA
:1038700088E0289F90011124929FA001939F500DF2
:10388000112470E0CA010E94D12E6038710540F405
:103890006115710519F406C068E070E0862F08957F
:1038A0008FE7089581E008958091EC0280FF08C0C1
:1038B0006091050170E0759567957595679521C0D4
:1038C00081FF06C06091050170E07595679519C08C
:1038D00082FF04C06091050170E010C09091EA027F
:1038E000992399F0609104019617A0F78091050142
:1038F000899FC001112470E00E94D12E60387105AB
:1039000040F46115710519F406C061E070E0862F7E
:1039100008958FE7089581E008958D3E21F40E9477
:10392000151C819504C08E3E29F40E94151C8093BD
:10393000F00208958F3E21F40E94151C819504C069
:10394000803F29F40E94151C8093EF020895893F5F
:1039500019F40E94541C05C08A3F31F40E94541C83
:1039600081958093F10208958B3F21F40E94541CAD
:10397000819504C08C3F29F40E94541C8093F2026C
:1039800008959FE0980F983078F421E030E0A90185
:1039900002C0440F551F9A95E2F7CA019091EE02BA
:1039A000892B8093EE0208958D3F21F48091EC02E3
:1039B00081600BC08E3F21F48091EC02826005C0D3
:1039C0008F3F29F48091EC0284608093EC0208958B
:1039D0008D3E39F49091F00297FF35C01092F002BD
:1039E00059C08E3E29F49091F0021916BCF32BC0F9
:1039F0009091EF028F3E29F497FF25C01092EF02BD
:103A000049C0803F19F41916CCF31DC09091F10202
:103A1000893F29F41916BCF41092F1023BC08A3F89
:103A200019F497FF10C0F8CF8B3F39F49091F20250
:103A300097FF09C01092F2022DC08C3F21F49091A3
:103A4000F2021916BCF39FE0980F983080F421E041
:103A500030E0A90102C0440F551F9A95E2F7CA0150
:103A600080959091EE0289238093EE0213C08D3FE2
:103A700021F48091EC028E7F0BC08E3F21F4809167
:103A8000EC028D7F05C08F3F29F48091EC028B7F83
:103A90008093EC028091EF02811106C08091F002C8
:103AA000811102C01092EB028091F102811106C0D7
:103AB0008091F202811102C01092EA020895809171
:103AC000E20283FF7EC081E794E00E94E2068091DB
:103AD000EE021F928F938CE694E09F938F930E9447
:103AE0007B078AE694E00E94E2068091EF02282F8D
:103AF000082E000C330B3F938F9387E694E09F933F
:103B00008F930E947B0785E694E00E94E2068091F5
:103B1000F002282F082E000C330B3F938F9382E680
:103B200094E09F938F930E947B0780E694E00E942D
:103B3000E2068091F102282F082E000C330B3F93F0
:103B40008F938DE594E09F938F930E947B078BE585
:103B500094E00E94E2068091F202282F082E000CC9
:103B6000330B3F938F9388E594E09F938F930E944C
:103B70007B0785E594E00E94E2068091EB021F92AC
:103B80008F9382E594E09F938F930E947B0780E55B
:103B900094E00E94E2068091EC021F928F938DE4E4
:103BA00094E09F938F930E947B078AE494E00E94A5
:103BB000E2068DB79EB74C960FB6F8949EBF0FBE27
:103BC0008DBF0E949A262091EF02211104C02091FE
:103BD000F002222321F09093E9028093E8022091E1
:103BE000F102211104C02091F202222321F09093CE
:103BF000E7028093E6028DEE92E00C94E424EF92CB
:103C0000FF920F931F93CF93DF9300D000D000D08B
:103C1000CDB7DEB786E0EDEEF2E0DE011196019061
:103C20000D928A95E1F7E090EF02F090F00200919A
:103C3000F1021091F2021092EF021092F002109233
:103C4000F1021092F202E11003C0FF2009F45DC0FE
:103C50008091E8029091E9020E94B226AC01909115
:103C6000EB02992339F020910A0130E0241735073F
:103C700058F04BC020910B018AE0289F900111243D
:103C80002417350718F041C09F3F19F09F5F9093AC
:103C9000EB02EE2061F00E94151C1E1414F09FEF41
:103CA00001C091E0989F902D11249093EF02FF2086
:103CB00061F00E94151C1F1414F09FEF01C091E0E9
:103CC000989F902D11249093F0023091EF023323AE
:103CD000E1F02091F0022223C1F045EB3403C00152
:103CE0001124992319F09093EF0203C081E080938F
:103CF000EF0235EB2303C0011124992319F09093AF
:103D0000F00203C081E08093F002011103C011238F
:103D100009F45DC08091E6029091E7020E94B2260C
:103D2000AC019091EA02992339F02091060130E02C
:103D30002417350758F04BC0209107018AE0289FCF
:103D4000900111242417350718F041C09F3F19F046
:103D50009F5F9093EA02002361F00E94541C1016AA
:103D600014F09FEF01C091E0989F902D1124909343
:103D7000F102112361F00E94541C111614F09FEF00
:103D800001C091E0989F902D11249093F202309100
:103D9000F1023323E1F02091F2022223C1F045EB3E
:103DA0003403C0011124992319F09093F10203C048
:103DB00081E08093F10235EB2303C00111249923A4
:103DC00019F09093F20203C081E08093F202809197
:103DD000EF0281110BC08091F002811107C0809128
:103DE000F102811103C08091F20281110E945F1DD6
:103DF000EB82FC820D831E8386E0FE013196ADEEE0
:103E0000B2E001900D928A95E1F726960FB6F894EC
:103E1000DEBF0FBECDBFDF91CF911F910F91FF90FD
:103E2000EF900895EDEEF2E086E0DF011D928A95B5
:103E3000E9F71092EB021092EA021092EC02089558
:103E4000CF93DF93EC01FB018281882309F43CC10D
:103E5000C430FDE5DF0760F4CB3F9CE5D90788F46B
:103E60009E0122503C452431310508F02EC109C085
:103E7000C236EDE5DE0729F0C63AFDE5DF0709F0B9
:103E800024C10E9484169093A1038093A003C131A2
:103E90008CE5D80709F4C6C008F042C0C930ECE58B
:103EA000DE0709F49BC000F5C5308CE5D80709F49E
:103EB00085C078F4C330ECE5DE0709F478C008F07B
:103EC0007AC0C230DC4509F0F5C08091A003816062
:103ED000EFC0C7309CE5D90709F478C008F07AC074
:103EE0008091A0038061E4C0CD30FCE5DF0709F4D8
:103EF00087C058F4CB309CE5D90709F479C008F0A5
:103F00007BC08091A00388606FC0CF30FCE5DF07E5
:103F100009F480C008F082C08091A003877FC8C0E8
:103F2000CE3F9CE5D90709F471C000F5C531FCE529
:103F3000DF0709F485C068F4C3319CE5D90709F4AB
:103F400075C008F095C00E941E108091A0038F7765
:103F5000AFC0CC3FFCE5DF07A9F108F054C0CB3F70
:103F6000DC4509F0A7C08091A10340C0C230EDE557
:103F7000DE0709F489C058F4C1158DE5D80709F4A6
:103F80005AC008F069C08091A10382602FC0C23678
:103F9000EDE5DE0709F47CC0C63AFDE5DF0709F46C
:103FA00081C0C330DD4509F085C080E06EC08091DE
:103FB000A00382607DC08091A00316C08091A00301
:103FC000886076C08091A10382604FC08091A00379
:103FD00080626EC08091A00380646AC00E941E103F
:103FE0008091A003806864C0846062C081603DC02D
:103FF0008091A0038E7F5CC08091A0038D7F58C00C
:104000008091A00316C08091A10318C08091A103E4
:104010008D7F2BC08091A0038F7E4AC08091A0032A
:104020008F7D46C08091A0038F7B42C08091A0030A
:10403000877F8B7F3DC08091A1038D7F8E7F15C0D0
:104040008091A00382FB222720F991E0922790FB28
:1040500082F990FB83F92CC08091A103982F909551
:1040600091708E7F892B90FB81F98093A10322C0F0
:104070000E941E108091A00387FB222720F991E067
:10408000922790FB87F914C081E00E941B1712C091
:104090008091A00384FB222720F991E0922790FBD6
:1040A00084F906C08091A003982F909590FB80F929
:1040B0008093A0038091A0039091A1030E94951684
:1040C0000E941E1080E001C081E0DF91CF91089531
:1040D000809104011F928F93809105011F928F930D
:1040E000809108011F928F93809109011F928F93F5
:1040F00080910A011F928F9380910B011F928F93E1
:1041000084E994E09F938F930E947B078DB79EB7BD
:104110000E960FB6F8949EBF0FBE8DBF08958832DD
:1041200020F58E3108F068C08B3091F1C0F48730F3
:1041300009F0BEC081E080930B0184E180930A0105
:104140008AE0809309018EE18093080188E08093E2
:10415000050188E28093040186EF95E0C6C08331B3
:1041600009F443C0843169F1A3C08F3409F49EC0BF
:1041700028F4893231F1883359F09AC0813531F011
:1041800008F4D4C0823509F4A7C092C08FEFA5C04F
:1041900088E196E00E94E2060E9468201F9281E07A
:1041A0008F931F9288E08F9381E195E09F938F9387
:1041B0000E947B070F900F900F900F900F900F9021
:1041C00096C085E196E00E94E2068091F70288237E
:1041D00009F4AAC01092F7021092F6021092F502AA
:1041E0001092F4021092F302B1C087E096E00E94B0
:1041F000E2060E9468207BC08D518093F7028330D5
:1042000031F170F48130D1F0823009F03FC08AE0A2
:1042100091E09093F6028093F5028CEC91E01FC040
:10422000853059F108F1863089F584E091E090936A
:10423000F6028093F50287E092E011C08BE091E0F6
:104240009093F6028093F50283EC91E008C089E038
:1042500091E09093F6028093F50288ED91E09093BF
:10426000F4028093F30218C088E091E09093F60284
:104270008093F50285EE91E0F2CF85E091E0909396
:10428000F6028093F50284EF91E0E9CF1092F702F5
:1042900084E096E00E94E2068091F702882309F408
:1042A00055C01F928F9380E096E00DC08AE015C044
:1042B00083EF95E01AC097FF47C0108280811F925C
:1042C0008F938DEE95E09F938F930E947B070F90C5
:1042D0000F900F900F900BC081E0E091F502F091EC
:1042E000F602309729F58AEE95E00E94E2062091C9
:1042F000F702222359F18091F3029091F402009782
:1043000011F48FEB91E09F938F931F922F9381EE87
:1043100095E09F938F930E947B070F900F900F90D3
:104320000F900F900F9016C080E0089586EFD5CFC4
:104330002081082E000C990B820F911D8F3F910553
:1043400009F00CF4B8CF8FEF8083B8CF8DED95E0F6
:104350000E94E20681E00895CF93C82F1F928F93A9
:104360008EE296E09F938F930E947B0781E090E01E
:10437000A0E0B0E0BC01CD0104C0660F771F881F2C
:10438000991FCA95D2F70E9476100F900F900F9048
:104390000F90CF910C941E10DF92EF92FF920F932B
:1043A0001F93CF93DF93482F50E0FA013597EF33F7
:1043B000F10508F03FC1E658FF4F0C94E52E0E942E
:1043C00080161F928F938EE79AE09F938F930E949F
:1043D0007B070E947C1683FB992790F91F929F937D
:1043E00082FB992790F91F929F9381FB992790F95F
:1043F0001F929F93982F91701F929F931F928F935C
:1044000085E39AE09F938F930E947B070E94841616
:1044100087FB222720F91F922F9386FB222720F962
:104420001F922F9385FB222720F91F922F9384FB45
:10443000222720F91F922F9383FB222720F91F9216
:104440002F9382FB222720F91F922F9391FB222783
:1044500020F91F922F93292F21701F922F9381FBF8
:10446000222720F91F922F93282F21701F922F931C
:104470009F938F9380E599E09F938F930E947B0792
:104480008DB79EB788960FB6F8949EBF0FBE8DBFAE
:1044900006C08EE39BE00E94E2060E941917C1E06D
:1044A000CEC08EE997E074C08091E202817F8E7F5A
:1044B0008093E20287E797E00E94E2068AE39BE0AE
:1044C0000E94E20681E08093F802E9CF8EE19BE052
:1044D0000E94E2060E94770BE2CF8091E202C82F91
:1044E000C095C170C0FB80F98093E202CC2319F023
:1044F00082E19BE091C085E09BE00E94E206809112
:10450000E202897F877F8093E202C9CF9091E20225
:1045100091FBCC27C0F981E0C827892FC0FB81F926
:104520008093E202CC2319F088EF9AE027C08AEE4C
:104530009AE02EC09091E20292FBCC27C0F981E074
:10454000C827892FC0FB82F98093E202CC2319F09F
:104550008BED9AE013C08BEC9AE01AC09091E202C6
:1045600093FBCC27C0F981E0C827892FC0FB83F9D2
:104570008093E202CC2351F08FEB9AE00E94E20696
:104580008091E20281608093E20259C082EB9AE05E
:104590000E94E20684CF87EB96E0FACF0E94A6261F
:1045A000062FF72EE82ED92EC091A003C7FBCC27EB
:1045B000C0F910912C03D09118010E948324DF923E
:1045C000EF92FF920F931F92CF931F921F931F9210
:1045D000DF931F928F9383E396E09F938F930E94C4
:1045E0007B078DB79EB70E960FB6F8949EBF0FBE91
:1045F0008DBF55CF0E941E109091A00397FBCC2732
:10460000C0F981E0C827892FC0FB87F98093A003F8
:10461000CC2329F088EA9AE00E94E20610C08DE9D6
:104620009AE0B6CF895303C08D5101C080E00E944B
:10463000AC2135CF8BE99AE00E94E206C0E08C2FD6
:10464000DF91CF911F910F91FF90EF90DF90089530
:1046500080E008950C942823CF93C82F8091F8020E
:10466000813071F040F0823009F045C08C2F0E94FB
:104670008F2081E046C00E9471158232F1F504C09E
:104680000E947115823261F48C2F0E942A238111BD
:1046900004C08C2F0E94CC212CC081E090E029C066
:1046A0008C2F0E942823811123C0C431C9F058F4F3
:1046B000CB3069F0C031B9F482E08093F80288E32E
:1046C0000E948F2015C0C93259F0C83361F487E7C2
:1046D00097E00E94E2068AE296E00E94E20608C0A5
:1046E0001092F8020CC088E296E00E94E20607C031
:1046F00081E0817006C01092F80280E002C080E084
:10470000F8CFCF910895CF93DF9386319C4541F543
:10471000EB010E947115982F8A812091020130913E
:104720000301882379F09A7A81E009F480E080938C
:10473000F902911102C069E201C065E3C9010E945A
:10474000D6250AC08091F902811102C069E201C038
:1047500065E3C9010E94E1250E94B61580E001C011
:1047600081E0DF91CF9108950F931F93CF93DF9353
:10477000C42FD22FFC0182818823C9F04093FC0210
:104780000E949A269093FB028093FA0280E28C0F9B
:10479000883008F057C0C77081E001C0880FCA9503
:1047A000EAF7DF91CF911F910F910C946D0D8091DD
:1047B000FC02481330C08091FA029091FB020E94E3
:1047C000B226883C910538F510E21D0FCD17B9F0DF
:1047D00080E28C0F883040F4C77081E001C0880F00
:1047E000CA95EAF70E94740D183028F581E09D2FD4
:1047F000977001C0880F9A95EAF70E946D0D802F7F
:104800000E94640D1830F0F4D77081E001C0880F69
:10481000DA95EAF70AC080E28C0F883098F4C77006
:1048200081E001C0880FCA95EAF7DF91CF911F910F
:104830000F910C94740D802FDF91CF911F910F91E8
:104840000C94640DDF91CF911F910F9108950F93F8
:104850009C01CB01243F4CE5340731F188F4293D1C
:10486000FCE53F07D9F02A3D4CE5340779F1283DB6
:104870003C45A9F506E221EE41EE68ED7CE52BC052
:10488000263FFCE53F07E1F0A8F0273F3C4539F51E
:1048900007E225EE46EE67EF7CE51DC007E225EE58
:1048A00045EE69ED7CE517C006E221EE40EE64EFCF
:1048B0007CE511C007E225EE44EE65EF7CE50BC018
:1048C00006E221EE42EE66EF7CE505C008E221E05B
:1048D00045EE6AED7CE50E94B42380E008C0FC014F
:1048E0008281882319F01092FC0201C081E00F91AF
:1048F000089590932D0280932C02089590930203C3
:10490000809301030895E0910103F0910203309731
:1049100021F00190F081E02D099480E00895EF925C
:10492000FF921F93CF93DF93FC01A0910103B091FD
:104930000203109709F442C080911801882341F0C6
:104940008091A00387FF04C08081818386E08083FB
:10495000EF011296ED91FC911397CE01099580918C
:10496000E20282FF2BC080FF04C087E59BE00E942B
:10497000E20618E081E5E82E8BE0F82E8091E20255
:1049800080FF0BC088811F928F93FF92EF920E944D
:104990007B070F900F900F900F90115021961111DF
:1049A000EDCF8091E20280FF09C08FE49BE0DF91B0
:1049B000CF911F91FF90EF900C94E206DF91CF9181
:1049C0001F91FF90EF900895E0910103F091020391
:1049D000309739F022E0DC012C930480F581E02D42
:1049E000099408952091FF02309100032817390798
:1049F00071F0909300038093FF02E0910103F09126
:104A00000203309721F00680F781E02D0994089584
:104A10002091FD023091FE022817390771F0909322
:104A2000FE028093FD02E0910103F09102033097B2
:104A300021F00084F185E02D09940895FC0132965F
:104A400080911801882331F08091A00387FF02C074
:104A50009EE101C096E080E0915028F02191222350
:104A6000D9F38F5FF9CF0895662351F12091180192
:104A70002223E9F02091A00327FF19C0462F469575
:104A8000469546954E31E0F4677021E030E002C073
:104A9000220F331F6A95E2F7FC01E40FF11D8281BA
:104AA00090E02823392381E0232B69F409C0FC011D
:104AB000329608962191621729F0E817F907D1F785
:104AC00080E0089581E008959C01FC0132969FEFFB
:104AD00080E04191461789F09F3F19F4411101C0D0
:104AE000982F8F5F8630A9F79F3F39F0F901E90FC2
:104AF000F11D97FDFA956283089508959C012A5F40
:104B00003F4FFC014281461301C012820196821779
:104B10009307B9F70895262F2695269526952E31C9
:104B200070F4FC01E20FF11D677021E030E001C07C
:104B3000220F6A95EAF78281282B228308958091BB
:104B4000E20280FF0CC01F926F9387E89BE09F9367
:104B50008F930E947B070F900F900F900F900895F6
:104B6000262F2695269526952E3178F4FC01E20F06
:104B7000F11D677021E030E001C0220F6A95EAF76D
:104B8000209582812823228308958091E20280FF6C
:104B90000CC01F926F9389E69BE09F938F930E94B6
:104BA0007B070F900F900F900F90089520911801A0
:104BB000222329F02091A00327FD0C948B250C942F
:104BC000642520911801222329F02091A00327FDBC
:104BD0000C94B0250C947E2520911801FC0132968E
:104BE000222331F08091A00387FF02C08EE101C033
:104BF00086E0DF011D928A95E9F7089508950C94E7
:104C0000FE2583E0809303030C94FF25811102C0ED
:104C100081E001C082E0809303030C94FF250C9493
:104C2000062681E0809303030C94FF250C94112643
:104C300008950C9418260C9419260C9418260C949C
:104C400018260C941826CF930E941F260E946C1BD6
:104C50000E941D26C0E08C2F0E94431A892B29F444
:104C6000CF5FC430C1F780E001C081E0CF910895EB
:104C700008951F920F920FB60F9211248F939F9356
:104C8000AF93BF9380910403811113C08091B2034D
:104C90009091B303A091B403B091B5034196A11DC7
:104CA000B11D8093B2039093B303A093B403B09368
:104CB000B503BF91AF919F918F910F900FBE0F9051
:104CC0001F9018958091BA03843031F10E94F70B40
:104CD0001092040320E488E190E00FB6F894A895C0
:104CE000809360000FBE2093600083B7817F846053
:104CF00083BF83B7816083BF7894889583B78E7FA5
:104D000083BF0FB6F894A895809160008861809366
:104D10006000109260000FBE08950E941E100C9457
:104D2000FB0B82E084BD93E095BD9AEF97BD809325
:104D30006E0008952FB7F8948091B2039091B30359
:104D4000A091B403B091B5032FBF08952FB7F89485
:104D50006091B2037091B3038091B4039091B50355
:104D60002FBF08959C014FB7F8948091B2039091A2
:104D7000B303A091B403B091B5034FBF821B930B53
:104D8000089578941F920F920FB60F9211248F936B
:104D90009F93AF93BF938091B2039091B303A0917F
:104DA000B403B091B5030196A11DB11D8093B20368
:104DB0009093B303A093B403B093B503BF91AF91A5
:104DC0009F918F910F900FBE0F901F901895F894A0
:104DD00081E08093E00080E28093D800E9ECF0E08D
:104DE00010828FE19EE40197F1F700C000001DBA28
:104DF000109268001CBC10BE1FBA10927A0010926C
:104E00006E0010926F00109271001092720010826A
:104E1000ECEBF0E0108214B817B81AB81DB810BA4D
:104E2000108215B818B81BB81EB811BA0C94003F00
:104E3000089580912B030895089522E02093E900BE
:104E40002FEF3091E800215035FD06C035ED3A9541
:104E5000F1F700002111F5CF2091E80025FF0BC0EC
:104E600040E050E066E070E00E941A2A8091E8007D
:104E70008E778093E8000895CF93DF9320911801F7
:104E8000222339F02091A00327FF03C060E222E033
:104E900002C068E021E02093E9002FEF3091E800A4
:104EA000215035FD06C035ED3A95F1F7000021118E
:104EB000F5CF2091E80025FF1DC0EC01809118017D
:104EC000811105C040E050E068E070E003C070E090
:104ED00040E050E0CE010E941A2A8091E8008E77CF
:104EE0008093E80080E2FE01ABE0B3E001900D9218
:104EF0008A95E1F7DF91CF9108958093070370932E
:104F00000903609308038091BA03843001F582E0BD
:104F10008093E9008FEF9091E800815095FD06C0E5
:104F200095ED9A95F1F700008111F5CF8091E80099
:104F300085FF0DC040E050E063E070E087E093E063
:104F40000E941A2A8091E8008E778093E8000895E5
:104F5000BC0184E00C947D27BC0183E00C947D2788
:104F600089EB9BE00E94E2068091B903811109C0A0
:104F70000E94AB2B0E94082C8091E20084608093F9
:104F8000E200089585EB9BE00E94E2061092B903CF
:104F9000089581EB9BE00E94E2060C9416268DEAB0
:104FA0009BE00E94E2066091B60381E0611101C0BE
:104FB00080E00C94012689EA9BE00E94E206909131
:104FC000BA0381E0943009F080E06091B6030C945C
:104FD0000626209106032F5F822F62E30E94B72EE0
:104FE000992319F0209306030895109206038091E7
:104FF0000A03882371F18091BA03843041F58091CE
:10500000E9008F702091EC00922F917020FD90E8C4
:10501000892B93E09093E9009091EB0090FF14C0EE
:105020009091EE0097FF10C09091E80095FF03C0AB
:105030001092F100F9CF9091E80090FF05C0909197
:10504000E8009E779093E8008F708093E9001092BB
:105050000A03089542E061EC81E00E94242B42E2C1
:1050600061EC82E00E94242B42E261EC83E00E942A
:10507000242B9091BA0381E0943009F080E0609194
:10508000B6030C940F268091BC03833009F461C0F1
:1050900030F4813071F0823009F49AC008958A307A
:1050A00009F486C08B3009F46CC0893009F0A8C0BF
:1050B00020C08091BB03813A09F0A2C08091E80032
:1050C000877F8093E8008091BF039091C003892B74
:1050D00021F460E28BE093E003C060E080E090E0C8
:1050E00070E00E94652A8091E8008B778093E80049
:1050F00008958091BB03813209F082C08091BF0383
:105100009091C003029708F07BC08091E800877FF0
:105110008093E8008091E80082FD05C08091BA0389
:105120008111F8CF6DC02091F3008091F20090E0E2
:10513000922B029731F48091F100813011F086308A
:1051400021F48091F10080932B038091E8008B770C
:1051500053C08091BB03813A09F052C08091BF03D4
:105160009091C003892B09F04BC08091E800877FA4
:105170008093E8008091E80080FFFCCF80911801C7
:1051800036C08091BB038132D9F58091BF039091E5
:10519000C003892BA9F58091E800877F8093E80000
:1051A0000E94592B8091BD03809318010C941E100E
:1051B0008091BB03813221F58091E800877F809345
:1051C000E8000E94592B8091BE0380932C03089520
:1051D0008091BB03813AA1F48091E800877F80939E
:1051E000E8008091E80080FFFCCF80912C03809341
:1051F000F1008091E8008E778093E8000C94592BA1
:1052000008959FB7F89410920A039FBF9091BA0334
:10521000943009F057C09091E9009F703091EC00F4
:10522000232F217030FD20E8922B23E02093E9000A
:105230002091EB0020FF43C02091EE0027FF3FC0EC
:1052400020910503222321F02091E80025FF37C09B
:105250001092050326E03091E80035FD15C030912D
:10526000BA03343061F53091EB0035FD28C0215090
:1052700021F481E08093050322C0EFE9FFE031973C
:10528000F1F700C00000E7CF8093F1008091E800C3
:1052900085FD0AC08091E80080FFFCCF8091E80086
:1052A0008E778093E80006C08FB7F89421E02093B2
:1052B0000A038FBF9F709093E90080E008959F706C
:1052C0009093E9008FEF089584B7877F84BF0FB66E
:1052D000F894A89580916000886180936000109296
:1052E00060000FBE90E080E80FB6F89480936100F4
:1052F000909361000FBE0C9411260E94AB2B0E946C
:10530000082CE2EEF0E080818460808378940C9435
:105310009C2E8CE091E00C947E248091BA03853021
:10532000C9F485EA9BE00E94E2068091BA038530C9
:1053300079F40E9462268091B8038823B1F30E9419
:105340002326882391F30E94042A0E941E10EDCF89
:105350000C948D26089508950C94AE29292F332797
:1053600023303105C9F060F42130310581F022305D
:10537000310509F041C08BE590E029EE3BE040C0EB
:1053800021323105E1F02232310531F135C082E1BF
:1053900090E024E43CE034C099278130910549F045
:1053A00028F0029749F5EDEBFBE005C0E5EEFBE0E8
:1053B00002C0EFECFBE0849190E09F0121C06330DC
:1053C0007105D0F4660F771FFB01EB5DFD4F208167
:1053D000318189E090E014C06330710568F4FB010D
:1053E000EE0FFF1FE15EFD4F20813181FB01E45E86
:1053F000FD4F808190E004C080E090E020E030E04C
:10540000FA0131832083089580E189BD82E189BD5D
:1054100009B400FEFDCF8091D8008F7D8093D80025
:105420008091E00082608093E0008091E00081FD47
:10543000FCCF0895CF92DF92EF92FF920F931F93CC
:10544000CF93DF93EC018B017A010E94782B8111BD
:1054500033C0E114F10439F0F70180819181081B18
:10546000190BC80FD91FC12CD12C0115110519F129
:105470008091E80085FD16C08091E8008E778093CA
:10548000E800E114F10449F0F70180819181C80E30
:10549000D91ED182C08285E00FC00E94782B88235C
:1054A00021F30AC089918093F10001501109FFEFA7
:1054B000CF1ADF0ADACF80E0DF91CF911F910F91F1
:1054C000FF90EF90DF90CF9008952091C10330912D
:1054D000C2032617370748F06115710539F420918A
:1054E000E8002E772093E80001C0B901FC0120E01C
:1054F0006115710579F18091BA038823F1F1853046
:10550000F1F18091E80083FD3CC08091E80082FDCC
:105510002EC08091E80080FFEBCF2091F3008091B6
:10552000F20090E0922B6115710551F088309105E1
:1055300038F421912093F100615071090196F3CF65
:1055400021E0089709F020E08091E8008E778093B1
:10555000E800CECF2111CFCF0AC08091BA038823B3
:1055600061F0853061F08091E80083FD0AC0809190
:10557000E80082FFF2CF80E0089582E0089583E0A2
:10558000089581E008952091C1033091C203261748
:10559000370748F06115710539F42091E8002E773E
:1055A0002093E80001C0B901FC0120E061157105FC
:1055B00091F18091BA03882309F440C0853009F441
:1055C0003FC08091E80083FD3DC08091E80082FDEE
:1055D0002FC08091E80080FFE9CF2091F3008091F7
:1055E000F20090E0922B6115710559F08830910519
:1055F00040F424912093F100319661507109019695
:10560000F2CF21E0089709F020E08091E8008E7742
:105610008093E800CBCF2111CCCF0AC08091BA0390
:10562000882361F0853061F08091E80083FD0AC035
:105630008091E80082FFF2CF80E0089582E0089533
:1056400083E0089581E00895982F973068F590934E
:10565000E900981739F07091EC002091ED0050911D
:10566000F00003C0242F762F50E021FD02C09F5F81
:10567000ECCF3091EB003E7F3093EB003091ED00AA
:105680003D7F3093ED003091EB0031603093EB00C3
:105690007093EC002093ED005093F0002091EE0009
:1056A00027FDE5CF80E008958F708093E90081E0C9
:1056B00008958091BB0387FF11C08091E80082FDAF
:1056C00005C08091BA038111F8CF11C08091E80024
:1056D0008B770BC08091BA03882349F08091E80052
:1056E00080FFF8CF8091E8008E778093E8000895DE
:1056F0002091E4003091E50095E64091EC00842F84
:10570000817040FF23C08091E80080FD1DC0809122
:10571000BA03882399F0853099F08091EB0085FDDC
:1057200011C04091E4005091E5002417350729F39A
:10573000915011F09A01E1CF84E0089582E008953C
:1057400083E0089581E0089580E008954091E800A5
:1057500042FFDDCF08950E94192C0E94212CE0EE1B
:10576000F0E0808181608083E8EDF0E080818F77D8
:10577000808319BCA7EDB0E08C918E7F8C938081E3
:105780008F7E80831092B90308950F931F93CF9358
:10579000DF930E94192C0E94212CC8EDD0E0888153
:1057A0008F77888388818068888388818F7D8883CC
:1057B00019BC1092BA031092B6031092B80310925B
:1057C000B70300EE10E0F80180818B7F8083888131
:1057D0008160888342E060E080E00E94242BE1EE5B
:1057E000F0E080818E7F8083E2EEF0E08081816056
:1057F0008083808188608083F80180818E7F8083B0
:10580000888180618883DF91CF911F910F910895E6
:10581000E8EDF0E080818F7E8083E7EDF0E080812D
:105820008160808384E082BF81E08093B9030C941F
:10583000C52BE8EDF0E080818E7F80831092E2003E
:1058400008951092DA001092E10008951F920F92CD
:105850000FB60F9211242F933F934F935F936F9343
:105860007F938F939F93AF93BF93EF93FF93809119
:10587000E10082FF0BC08091E20082FF07C08091AF
:10588000E1008B7F8093E1000E94E9278091DA009C
:1058900080FF1FC08091D80080FF1BC08091DA007C
:1058A0008E7F8093DA008091D90080FF0DC080E167
:1058B00089BD82E189BD09B400FEFDCF81E08093FE
:1058C000BA030E94B02705C019BC1092BA030E9407
:1058D000C2278091E10080FF19C08091E20080FF23
:1058E00015C08091E2008E7F8093E2008091E200FB
:1058F00080618093E2008091D80080628093D8001C
:1059000019BC85E08093BA030E94CF278091E10003
:1059100084FF30C08091E20084FF2CC080E189BD0B
:1059200082E189BD09B400FEFDCF8091D8008F7D52
:105930008093D8008091E1008F7E8093E100809178
:10594000E2008F7E8093E2008091E200816080938C
:10595000E2008091B603882311F084E007C08091B3
:10596000E30087FD02C081E001C083E08093BA03B9
:105970000E94DB278091E10083FF29C08091E20033
:1059800083FF25C08091E100877F8093E10082E062
:105990008093BA031092B6038091E1008E7F8093CA
:1059A000E1008091E2008E7F8093E2008091E2002E
:1059B00080618093E20042E060E080E00E94242B5E
:1059C0008091F00088608093F0000E94C927FF91C9
:1059D000EF91BF91AF919F918F917F916F915F9167
:1059E0004F913F912F910F900FBE0F901F901895E0
:1059F0001F920F920FB60F9211242F933F934F9344
:105A00005F936F937F938F939F93AF93BF93CF9346
:105A1000DF93EF93FF93C091E900CF708091EC008A
:105A2000D82FD17080FDD0E81092E9008091F0006D
:105A3000877F8093F00078940E943C2D1092E900BB
:105A40008091F00088608093F000CD2BCF70C093E0
:105A5000E900FF91EF91DF91CF91BF91AF919F91BD
:105A60008F917F916F915F914F913F912F910F9007
:105A70000FBE0F901F9018951F93CF93DF93CDB754
:105A8000DEB7AA970FB6F894DEBF0FBECDBFEBEB23
:105A9000F3E08091F100819323E0E33CF207C9F742
:105AA0000E9443288091E80083FF2EC18091BB03B0
:105AB0009091BC03492F50E04A30510508F024C1B1
:105AC000FA01E754FF4F0C94E52E803821F082381C
:105AD00009F01AC108C08091B7039091B8039923C7
:105AE00089F082600FC08091BF038F70873008F00B
:105AF0000BC18093E9008091EB0085FB882780F93A
:105B00001092E9009091E800977F9093E8008093CD
:105B1000F1001092F100D1C0282F2D7F09F0F4C0C0
:105B2000882319F0823061F0EFC08091BD0381308D
:105B300009F0EAC0933009F080E08093B8032EC0EA
:105B40008091BD0381112AC08091BF038F702FEF18
:105B5000280F263008F0D8C08093E9002091EB0090
:105B600020FF1CC0933021F48091EB00806214C0B0
:105B70009091EB0090619093EB0021E030E0A9015F
:105B800002C0440F551F8A95E2F74093EA00109235
:105B9000EA008091EB0088608093EB001092E900AE
:105BA0008091E800877F8093E8000E94592BACC069
:105BB0008111AAC01091BD031F778091E300807806
:105BC000812B8093E3008091E800877F8093E80039
:105BD0000E94592B8091E80080FFFCCF8091E30068
:105BE00080688093E300111102C082E001C083E06D
:105BF0008093BA0389C08058823008F085C08091B4
:105C0000BD039091BE038C3D53E0950779F583E089
:105C10008A838AE289834FB7F894DE01139620E0E5
:105C20003EE051E2E32FF0E050935700E49120FF73
:105C300003C0E295EF703F5FEF708E2F90E0EA3087
:105C400010F0C79601C0C0968D939D932F5F2431AD
:105C500049F74FBF8091E800877F8093E8006AE2B0
:105C600070E0CE0101960E94652A16C06091BF03C4
:105C70007091C003AE014F5F5F4F0E94AC29BC0121
:105C8000892B09F441C09091E800977F9093E80038
:105C900089819A810E94C32A8091E8008B77809342
:105CA000E80032C0803881F58091E800877F8093DA
:105CB000E8008091B6038093F1008091E8008E7730
:105CC00072CF811121C08091BD039091BE039927AD
:105CD0000297D4F48091E800877F8093E800809158
:105CE000BD038093B6030E94592B8091B6038111A6
:105CF00006C08091E30087FD02C081E001C084E01E
:105D00008093BA030E942A288091E80083FF0AC08A
:105D10008091E800877F8093E8008091EB008062AB
:105D20008093EB00AA960FB6F894DEBF0FBECDBFEE
:105D3000DF91CF911F910895CF938091BA0388236B
:105D4000A1F0C091E900CF709091EC00892F817093
:105D500090FD80E8C82B1092E9008091E80083FD57
:105D60000E943C2DCF70C093E900CF910895991BFC
:105D700079E004C0991F961708F0961B881F7A9542
:105D8000C9F78095089587FB082E062687FD819523
:105D900067FD61950E94B72E0EF4919507FC8195E1
:105DA000089597FB072E16F4009407D077FD09D0CD
:105DB0000E94EB2E07FC05D03EF4909581959F4FF5
:105DC0000895709561957F4F0895EE0FFF1F059020
:105DD000F491E02D0994AA1BBB1B51E107C0AA1F37
:105DE000BB1FA617B70710F0A61BB70B881F991F7C
:105DF0005A95A9F780959095BC01CD010895FB01B6
:105E0000DC0104C08D910190801921F44150504073
:105E1000C8F7881B990B0895F999FECF92BD81BDF3
:105E2000F89A992780B50895A8E1B0E042E050E0E3
:105E30000C94402F262FF999FECF92BD81BDF89A80
:105E4000019700B4021639F01FBA20BD0FB6F894BE
:105E5000FA9AF99A0FBE08950396272F0E941B2FD6
:105E60000E941A2F252F0E941B2F242F0C941B2FCA
:105E70000196272F0E941B2F0C941A2FDC01CB01B7
:105E8000FC01F999FECF06C0F2BDE1BDF89A31964A
:105E900000B40D9241505040B8F70895F894FFCFE8
:105EA000C800B002280850011E0A140119273C2717
:105EB0001D27AC27A8271C270170726F63657373B9
:105EC0005F7265636F72645F757365720070617293
:105ED00073655F6E65787400657865637574655F7A
:105EE000686561645F616E645F706F7000E200E915
:105EF00000EA00B500B600B700CD008301CC008AEF
:105F00000192019401210223022402250226022784
:105F1000022A02B300B4006F007000818283E200A5
:105F2000E900EA00B500B600B700CD008301CC005F
:105F30008A019201940121022302240225022602F1
:105F400027022A02B300B4006F00700081828366CA
:105F50009392919037F6F73635349730F032F43F1C
:105F60003F3F006D6B5F64656C6179006D6B5F69CD
:105F70006E74657276616C006D6B5F6D61785F73D6
:105F800070656564006D6B5F74696D655F746F5FEC
:105F90006D6178006D6B5F776865656C5F6D6178CA
:105FA0005F7370656564006D6B5F776865656C5FD6
:105FB00074696D655F746F5F6D61780040B6222E05
:0C5FC0000D780C560CFB0B140C2D0C0083
:00000001FF
